:020000040000FA
:040000006C303A28FE
:08000800A000030EA100831209
:100010008B1C32288B1031181428B11C3228643004
:10002000010203183128182800001628172818285C
:1000300019281A281B281C281D281E281F283110A3
:10004000B114A810031005190314AA0DA90DA80DC9
:10005000B00B322831152A08AF002908AE00280855
:10006000AD00B11081010B11210E8300A00E200EF6
:02007000090085
:0C007400203084008001840A6030040207
:10008000031C3C281230B000A22183160C308505D9
:1000900087018312850187010730990000309A009B
:1000A000103083168E008312603083168F00831207
:1000B0000030831691008312C830831681008312AA
:1000C00031309000003083168C00831210308B008A
:1000D000831600309B001C141A088312BC00851D77
:1000E000E621831610309B001C141A088312BD00F1
:1000F000DE2181018E018F010B118B100B108C0101
:100100008B1790203119A620B30B8E280310851968
:100110000314B90DF030390203191F210B22812875
:100120006400311808000B1D08000B11B1103114C8
:100130001230B000051DA12832148316011383125A
:1001400008003210831601178312080031110130A4
:10015000B7008B132030370783169B001C141A0836
:100160008312A400A500C030A506103037078316FF
:100170009B001C141A088312A30000303707831653
:100180009B001C141A088312A2008B17321CCE2865
:1001900022090339A200A309A409A50922082D02F6
:1001A000031D192923082E02031D192924082F02D3
:1001B000031D192901303702031DE3283D18E328E8
:1001C0003D143E14AE2102303702031DEC28BD1849
:1001D000EC28BD143E14B02103303702031DF5286E
:1001E0003D19F5283D153E14B22104303702031D98
:1001F000FE28BD19FE28BD153E14B4210530370276
:10020000031D07293D1A07293D163E14B621063065
:100210003702031D1029BD1A1029BD163E14B8213E
:1002200007303702031D19293D1B19293D173E14BC
:10023000BA21B70A0830370203180800A92801308C
:10024000B600B300B400B500B70085018701B11353
:100250009020B30B5329031085190314B90DF03006
:10026000390203197A29B40B5329013037020319D3
:10027000C521023037020319CA210330370203199E
:10028000CD21043037020319D0210530370203197C
:10029000D521063037020319D82107303702031958
:1002A000DB219630B400311D28293111321C5D2923
:1002B0002D090339AD00AE09AF092F1CB1132F1C56
:1002C0002829B11B28292E182829B1178B13203073
:1002D0003707BB002F08BA008D2110303707BB004D
:1002E0002E08BA008D2100303707BB002D08BA0058
:1002F0008D218B1785018701B70AB60108303702B7
:10030000031C2829DE2108003E1C08003E10103086
:10031000BB003D08BA008D2108008B133A088316F4
:100320001C159A0083123B0883169B0055309D00D4
:10033000AA309D009C1464009C189B291C118312F8
:100340008B170800FF30D000D415D515D615D7155A
:10035000D815D915DA15DB15DC150800F130BD29E3
:10036000F230BD29F430BD29F830BD291F30C12934
:100370002F30C1294F30C1290800BD050F30D204EC
:100380000800BD05F030D2040800103085060230A8
:100390008706080020308506080021308506080001
:1003A00002308506023087060800183087060800EC
:1003B0002130870608000930870608003D08D20072
:1003C000031D08001130BD00D2000800B601B301C2
:1003D000B4013C1CEE29BC01BC14F029BC013C1446
:1003E0003C08B6006400F429F529F629F729F82914
:1003F000B41B0516B41F0512B30BF229B40BF22976
:100400000310B60CB608031DF2290030BB003C08EF
:10041000BA008D2108008F08031908008F01D00F42
:10042000462BD00A0E305205031D252A541D1B2AC7
:10043000D4015416332AD41D202AD4015416332A49
:10044000541E332AD401D414332AD41C2A2AD401AA
:100450005415332A541D2F2AD401D415332A541E7F
:10046000332AD401541509305205031D462A551D5F
:100470003C2AD5015516542AD51D412AD5015516B9
:10048000542A551E542AD501D514542AD51C4B2A5A
:10049000D5015515542A551D502AD501D515542A74
:1004A000551E542AD50155150B305205031D672AD8
:1004B000561D5D2AD6015616752AD61D622AD6010A
:1004C0005616752A561E752AD601D614752AD61CBC
:1004D0006C2AD6015615752A561D712AD601D615D5
:1004E000752A561E752AD601561507305205031D6A
:1004F000882A571D7E2AD7015716962AD71D832A88
:10050000D7015716962A571E962AD701D714962A2E
:10051000D71C8D2AD7015715962A571D922AD70125
:10052000D715962A571E962AD70157150630520519
:10053000031DA92A581D9F2AD8015816B72AD81D6D
:10054000A42AD8015816B72A581EB72AD801D81499
:10055000B72AD81CAE2AD8015815B72A581DB32A75
:10056000D801D815B72A581EB72AD8015815103007
:10057000BC1819305205031DCC2A591DC22AD901B5
:100580005916DA2AD91DC72AD9015916DA2A591E4D
:10059000DA2AD901D914DA2AD91CD12AD901591554
:1005A000DA2A591DD62AD901D915DA2A591EDA2A8A
:1005B000D90159155030BC1859305205031DEF2A86
:1005C0005A1DE52ADA015A16FD2ADA1DEA2ADA014D
:1005D0005A16FD2A5A1EFD2ADA01DA14FD2ADA1CFF
:1005E000F42ADA015A15FD2A5A1DF92ADA01DA1518
:1005F000FD2A5A1EFD2ADA015A156030BC186930EE
:100600005205031D122B5B1D082BDB015B16202BF3
:10061000DB1D0D2BDB015B16202B5B1E202BDB0172
:10062000DB14202BDB1C172BDB015B15202B5B1D48
:100630001C2BDB01DB15202B5B1E202BDB015B154C
:100640002030BC1829305205031D352B5C1D2B2B87
:10065000DC015C16432BDC1D302BDC015C16432BCC
:100660005C1E432BDC01DC14432BDC1C3A2BDC012D
:100670005C15432B5C1D3F2BDC01DC15432B5C1E02
:10068000432BDC015C1584213D08D2005008D100C9
:100690000C305405031D05120C305505031D851241
:1006A0000C305605031D05100C305705031D851031
:1006B0000C305805031D87100C305905031D071019
:1006C0000C305A05031D87120C305B05031D071201
:1006D0000C305C05031D871151080E020318982B7E
:1006E00012305405031D051612305505031D8516DD
:1006F00012305605031D051412305705031D8514CD
:1007000012305805031D871412305905031D0714B4
:1007100012305A05031D871612305B05031D07169C
:1007200012305C05031D8715FF30500203190800C5
:100730008F08031D0800902051080E02031C982BFF
:1007400018305405031D051206305405031D051607
:1007500018305505031D851206305505031D8516F5
:1007600018305605031D051006305605031D0514E7
:1007700018305705031D851006305705031D8514D5
:1007800018305805031D871006305805031D8714BF
:1007900018305905031D071006305905031D0714AD
:1007A00018305A05031D871206305A05031D871697
:1007B00018305B05031D071206305B05031D071685
:1007C00018305C05031D871106305C05031D871575
:0207D00008001F
:084000000A00030002000600A3
:02400E00CC33B1
:10420000010003000300030003000200020002009B
:1042100002000000000000000000FF00FF00FF009F
:10422000000000000000000000000000000000008E
:104230000000C000C000C000C000FF00FF00FF0081
:104240000100C300F300CF00FF00C300F300CF0064
:10425000FF00C300F300CF00FF00FF00FF00FF00DE
:10426000FF00FF00FF00FF00FF00FF00FF00FF0056
:10427000FF00FF00FF00FF00FF00FF00FF00FF0046
:10428000FF00FF00FF00FF00FF00FF00FF00FF0036
:10429000FF00FF00FF00FF00FF00FF00FF00FF0026
:1042A000FF00FF00FF00FF00FF00FF00FF00FF0016
:1042B000FF00FF00FF00FF00FF00FF00FF00FF0006
:1042C000FF00FF00FF00FF00FF00FF00FF00FF00F6
:1042D000FF00FF00FF00FF00FF00FF00FF00FF00E6
:1042E000FF00FF00FF00FF00FF00FF00FF00FF00D6
:1042F000FF00FF00FF00FF00FF00FF00FF00AA001B
:00000001FF
